:020000040000fa
:08000000407f04000100000034
:020000040000fa
:1002000000000000000000000000000000000000ee
:1002100000000000000000000000000000000000de
:1002200000000000000000000000000000000000ce
:1002300000000000000000000000000000000000be
:020000040002f8
:10fe8000af88200060792200000188000000000097
:10fe900000002800b010880000402000c01088003a
:10fea00030002000f0108800048020002f000700a0
:10feb000114cb1003a003a0012c7b300d2108800ca
:10fec000b2c4b300d21088008006eb00048020008a
:10fed00046002000250007000603e900fdff3a0068
:10fee0000c4080001340800093018800160620001b
:10fef0001e0007000603e900fdff3a000d00e000c8
:10ff000003003200e2c4b300d2108800eeff3700d5
:10ff1000000ebb00100424000060fe000a00070071
:10ff2000448020001f00080003000000345ebb0076
:10ff30003456bb0034cebb000c86e8001000240011
:10ff400001000700deff3700003b8800500520005d
:10ff5000303b8800a00a2000303b880061e7a80001
:10ff60000000000000000000000006001a01200050
:10ff70000b0020001802ae0004003700e1108000e2
:10ff8000015a78008dc64000000006000060fe00a7
:10ff90008b05e900f7ff3a000a05e900f4ff3a0093
:10ffa0001622ef00b2ff37004d65000073610000bc
:04ffb0006a210000c2
:020000040000fa
:020000040002f8
:10ffb400000800008a0000000000000000000000ab
:020000040000fa
:0200000401f009
:04000000f5ff000008
:020000040000fa
:0200000401f009
:04000400ff7f00007a
:020000040000fa
:0200000401f009
:040008007fff000076
:020000040000fa
:0200000401f009
:04001400ffff0000ea
:020000040000fa
:10000800e27f0100e27f0100e27f0100e27f010060
:10001800e27f0100e27f0100e27f0100e27f010050
:10002800e27f0100e27f0100e27f0100e27f010040
:10003800e27f0100e27f0100e27f0100e27f010030
:10004800e27f0100e27f0100e27f0100e27f010020
:10005800e27f0100e27f0100e27f0100e27f010010
:10006800e27f0100e27f0100e27f0100e27f010000
:10007800e27f0100e27f0100e27f0100e27f0100f0
:10008800e27f0100e27f0100e27f0100e27f0100e0
:10009800e27f0100e27f0100e27f0100e27f0100d0
:1000a800e27f0100e27f0100e27f0100e27f0100c0
:1000b800e27f0100e27f0100e27f0100e27f0100b0
:1000c800e27f0100e27f0100e27f0100e27f0100a0
:1000d800e27f0100e27f0100e27f0100e27f010090
:1000e800e27f0100e27f0100e27f0100e27f010080
:0800f800e27f0100e27f01003c
:020000040000fa
:10010800e27f0100e27f0100e27f0100e27f01005f
:10011800e27f0100e27f0100e27f0100e27f01004f
:10012800e27f0100e27f0100e27f0100e27f01003f
:10013800e27f0100e27f0100e27f0100e27f01002f
:10014800e27f0100e27f0100e27f0100e27f01001f
:10015800e27f0100e27f0100e27f0100e27f01000f
:10016800e27f0100e27f0100e27f0100e27f0100ff
:10017800e27f0100e27f0100e27f0100e27f0100ef
:10018800e27f0100e27f0100e27f0100e27f0100df
:10019800e27f0100e27f0100e27f0100e27f0100cf
:1001a800e27f0100e27f0100e27f0100e27f0100bf
:1001b800e27f0100e27f0100e27f0100e27f0100af
:1001c800e27f0100e27f0100e27f0100e27f01009f
:1001d800e27f0100e27f0100e27f0100e27f01008f
:1001e800e27f0100e27f0100e27f0100e27f01007f
:0801f800e27f0100e27f01003b
:020000040000fa
:020000040002f8
:04ffc4000000fe003b
:00000001FF
